:020000040000FA
:1000000048201F30850007309F0045200030A000A9
:100010004520201C3620452020180F200828452088
:10002000201D26204520201D08002108A200362082
:10003000452020182E20452020180800A01D08006B
:10004000210E2204A1002011A0110800452005085E
:100050000F394520A1002010201508004520050873
:100060000F394520A1002010A01508004520A01838
:100070003E284520051E08004520A0144520051AED
:1000800008004520A0102014080003138312080064
:10009000031383160800031783120800031783163F
:0200A000080056
:02400E00F13F80
:00000001FF
